:100000003AC053C052C051C06BC14FC04EC04DC06A
:10001000A7C04BC04AC049C048C047C046C045C041
:1000200044C044C042C0B8C0B9C0BAC0BBC0BCC064
:10003000BDC0BEC0BFC0C0C0C1C0C2C0C3C0C4C0BC
:10004000C5C0C6C0C7C0C8C0C9C0CAC0CBC013C124
:1000500014C115C116C117C118C119C11AC11BC1DC
:100060001CC11DC11EC11FC120C121C122C123C18C
:1000700024C125C126C111241FBECFE5D4E0DEBFB7
:10008000CDBF10E0A0E6B0E0ECE9F3E002C00590DF
:100090000D92A236B107D9F710E0A2E6B0E001C098
:1000A0001D92A33EB107E1F74DC1AACF1F920F9257
:1000B0000FB60F9211248F939F93EF93FF9381B10B
:1000C0009927803A910599F1813A91058CF4883607
:1000D000910569F18936910524F48036910539F14D
:1000E00036C080389105A9F08838910591F02FC06D
:1000F000803B9105F1F0813B910524F4883A91050C
:10010000C1F025C0883B910591F0803C9105F9F440
:100110000EC0E0916100E7FD07C0FF27ED59FF4FDA
:1001200083B1808380E801C083B18093610085EC56
:100130000DC0E0916100E7FD08C0FF27ED59FF4FBA
:10014000808183B980E88093610085E886BFFF9154
:10015000EF919F918F910F900FBE0F901F90189568
:100160001F920F920FB60F9211242F933F934F932C
:100170008F939F93AF93BF93EF93FF932091620070
:10018000822F9927AA27BB27FC013197E431F1057B
:1001900050F5ED5EFF4F0994909825C0919823C0CB
:1001A000929821C093981FC094981DC0C6981BC0F8
:1001B000C79819C0959817C0969815C0979813C0FE
:1001C000C09811C0C1980FC0C2980DC0C3980BC091
:1001D000C49809C0C59807C0A89805C0A99803C0CD
:1001E000AA9801C0AB98822F8F5F809362008531FF
:1001F00058F490916200E92FFF27ED59FF4F80815D
:10020000882381F4892FF0CF80916000882331F01A
:1002100081E0809362008093600004C08EBD809373
:10022000620050C0809179009927982F88272091EB
:100230007A00820F911D22273327281B390B40910A
:100240006200E42FFF27ED59FF4F908180917800E5
:10025000989FC0011124281B390B3DBD2CBD842F54
:100260009927AA27BB27FC013197E431F10550F506
:10027000E95DFF4F0994909A25C0919A23C0929A04
:1002800021C0939A1FC0949A1DC0C69A1BC0C79ADA
:1002900019C0959A17C0969A15C0979A13C0C09A1C
:1002A00011C0C19A0FC0C29A0DC0C39A0BC0C49AA4
:1002B00009C0C59A07C0A89A05C0A99A03C0AA9AFE
:1002C00001C0AB9AFF91EF91BF91AF919F918F9138
:1002D0004F913F912F910F900FBE0F901F90189547
:1002E0001F920F920FB60F9211248F939F938EB58A
:1002F000992787709070892B11F01092600081E02F
:100300008EBD80917B0084BD9F918F910F900FBE19
:100310000F901F90189580E0E82FFF27ED59FF4FB1
:1003200010828F5F87FFF8CF81E0809363008FE1B9
:10033000809378008093790080E480937A00109213
:100340007B000895CFE5D4E0DEBFCDBFE4DF8FEFC3
:1003500087BB84BB81BB18BA15BA12BA11B880E248
:1003600080B982EC82B985E486BF85E085BD809145
:100370007B0084BD1EBC89B7846489BF789485B72F
:100380008F7885BF80916300813009F0C4DF85B725
:0C039000806885BF889585B78F77F3CF14
:02039C000180DE
:00000001FF
